:1000000005308A00D02D00008E30A0003A08A100F3
:100010003908A200A301A108031D18282208A10085
:10002000A2010830A002A108031D1828A001202861
:100030000310A11B1F28A20DA10DA0031828A113B6
:10004000080039080319E628C5003D080319E62809
:10005000C502031C30287F30C5070318E628362860
:100060008130C502031CE6280319E6284508A000D4
:10007000A101A201A301C4013A08C300C3173B08B0
:10008000C2003C08C1001930C5004008C102031875
:1000900059280130C20203185928C30203185928ED
:1000A000C40203185928C40AC30AC20A4008C10777
:1000B0008B283F08C202031874280130C3020318BA
:1000C0007428C40203187428C40AC30A3F08C2076C
:1000D0004008C107031C8B28C20A031D8B28C30AD2
:1000E000031D8B28C40A8B283E088038C3020318DE
:1000F0008A280130C40203188A28C40A3E088038BE
:10010000C3073F08C207031C6828C30A031D6828E9
:10011000C40A68282314C50B8E2899280310C10D22
:10012000C20DC30DC40D0310A30DA20DA10DC60D6C
:100130004528461CA1280310A10CA20CA30CC60C38
:10014000A428A0030319E628C61BCD280310C10D5F
:10015000C20DC30DC40D4008C1020318B9280130F7
:10016000C2020318B928C3020318B928C402031C29
:10017000DC283F08C2020318C4280130C302031858
:10018000C428C402031CDC283E088038C3020318BC
:10019000CD280130C402031CDC28A30A031DDC287F
:1001A000A20A031DDC28A10A031DDC28A00A0319EA
:1001B000E628A10CA20CA30C3A08C5003E08C5060F
:1001C000C51FE428A117EA28A113EA28A001A1016C
:1001D000A201A30108008E30A0003708A002380851
:1001E000A2003908A100A217A008031902290310D0
:1001F000A208031DFE28A10803190229A20CA10CC4
:10020000A00BF728B81F0929A109A209A10A0319FF
:10021000A20A08000030A1001F08C73921049F006E
:100220002030A000A00B1229152900001F151F194E
:1002300017291E08A30083161E088312B7001E0884
:10024000B800BA003708B90004202308BC0022080F
:10025000BB002108BA002008B9003330C000BF003D
:10026000BE008030BD0021202308BA002208B9005A
:100270002108B8002008B700EB202208A6002108BA
:10028000A5000830A1001F08C73921049F002030B5
:10029000A000A00B49294C2900001F151F194E2949
:1002A0001E08A30083161E088312B7001E08B8009C
:1002B000BA003708B90004202308BC002208BB009C
:1002C0002108BA002008B9003330C000BF00BE00CA
:1002D0008030BD0021202308BA002208B90021087F
:1002E000B8002008B700EB202208A8002108A700CA
:1002F0002608003C03188729FF3A031D8329250897
:10030000683C031887290130A6006830A50028083A
:10031000003C03189629FF3A031D92292708683CE0
:10032000031896290130A8006830A7008A11E62D2D
:10033000A101A201A001A3014408031DA2294308B1
:100340000319BC291030C5000310C10DC20DA00D4A
:10035000A30D44082302031DAF2943082002031CF8
:10036000B8294308A002031CA3034408A3020314F2
:10037000A10DA20DC50BA4290800A001A1014208EE
:1003800003104318A007A00CA10CC318A007A00CD1
:10039000A10C4319A007A00CA10CC319A007A00C25
:1003A000A10C431AA007A00CA10CC31AA007A00C13
:1003B000A10C431BA007A00CA10CC31BA007A00C01
:1003C000A10C08004208A10141020318EA294108D2
:1003D000A000F629A0010830C300C10DA00D4208FD
:1003E00020020318A000A10DC30BED290800023064
:1003F000B7009E30B8002430B9000C30BA009830F5
:10040000BB004830BC00C030BD001E30BE00BF0184
:100410001830C0002808C2002708C100C401643099
:10042000C30098212108AF002F08C2006430C30028
:10043000BD2121082702B0003008C1000A30C200E7
:10044000E2212108C1000A30C2002108C300BD21F9
:1004500021083002B1003008C1000A30C200E22198
:100460002108B0002608C2002508C100C40164307C
:10047000C30098212108AC002C08C2006430C300DE
:10048000BD2121082502AD002D08C1000A30C2009F
:10049000E2212108C1000A30C2002108C300BD21A9
:1004A00021082D02AE002D08C1000A30C200E22151
:1004B0002108AD0037302F0784000008AF00373027
:1004C000300784000008B00037303107840000088E
:1004D000B10037302C0784000008AC0037302D07FE
:1004E00084000008AD0037302E0784000008AE00FD
:1004F0008316860183123108860083160610831244
:1005000006148316061083120610831686018312C2
:100510003008860083168813831288178316881381
:10052000831288138316860183122F088600831690
:1005300008138312081783160813831208138316EF
:10054000860183122E08860083168812831288166D
:1005500083168812831288128316860183122D084F
:100560008600831608128312081683160812831257
:1005700008128316860183122C0886008A11E72D43
:100580008316A0010430A1000830A2000D30A300A2
:100590001130A4001630A5001A30A6001F30A700A5
:1005A0002330A8002730A9002C30AA003030AB003F
:1005B0003530AC003930AD003D30AE004130AF00D9
:1005C0004630B0004A30B1004E30B2005330B30074
:1005D0005730B4005B30B5005F30B6006330B70011
:1005E0006730B8006B30B9006F30BA007330BB00B1
:1005F0007730BC007B30BD007F30BE008330BF0051
:100600008730C0008A30C1008E30C2009230C300F3
:100610009530C4009930C5009C30C600A030C7009A
:10062000A330C800A730C900AA30CA00AD30CB0043
:10063000B130CC00B430CD00B730CE00BA30CF00EE
:10064000BD30D000C030D100C330D200C630D3009E
:10065000C830D400CB30D500CE30D600D030D70053
:10066000D330D800D530D900D830DA00DA30DB000A
:10067000DC30DC00DF30DD00E130DE00E330DF00C5
:10068000E530E000E730E100E830E200EA30E30086
:10069000EC30E400EE30E500EF30E600F130E7004A
:1006A000F230E800F330E900F530EA00F630EB0014
:1006B000F730EC00F830ED00F930EE00FA30EF00E2
:1006C000FB30F000F100FC30F200FD30F300F400EC
:1006D000FE30F500F600F700F800F900FF30FA00F0
:1006E00083122808013C031C8A2B031D7B2B27083F
:1006F000683C031C8A2B2708683CB7000130B8000F
:100700002808031C280FB802A0303707840000080F
:10071000B40036112808013C031CA32B031D942BA5
:1007200027080E3C031CA32BB4302702B70028086F
:10073000B8000030031C0130B802A0303707840035
:100740000008B4003611A808031DB82B2708B43CD4
:10075000031CB82B2708B43CB700B8012808031CB9
:10076000280FB802A030370784000008B4003615FF
:10077000A808031DC52B27085A3C031CC52BA03015
:10078000270784000008B40036152808013C031C24
:10079000DE2B031DCF2B2708683C031CDE2B0E30FD
:1007A0002702B7002808B8000130031C0230B80245
:1007B000A030370784000008B500B6152808013CB2
:1007C000031CF72B031DE82B27080E3C031CF72BFB
:1007D00027080E3CB7000130B8002808031C280F7A
:1007E000B802A030370784000008B500B611A80889
:1007F000031D0D2C2708B43C031C0D2C5A30270276
:10080000B7002808B8000030031C0130B802A0303F
:10081000370784000008B500B611A808031D222C74
:1008200027085A3C031C222C27085A3CB700B80161
:100830002808031C280FB802A030370784000008DE
:10084000B500B6152608013C031C3B2C031D2C2CBF
:100850002508683C031C3B2C2508683CB700013088
:10086000B8002608031C260FB802A0303707840002
:100870000008B20036102608013C031C542C031D4E
:10088000452C25080E3C031C542CB4302502B7001F
:100890002608B8000030031C0130B802A03037072A
:1008A00084000008B2003610A608031D692C250834
:1008B000B43C031C692C2508B43CB700B8012608D9
:1008C000031C260FB802A030370784000008B200CE
:1008D0003614A608031D762C25085A3C031C762CDA
:1008E000A030250784000008B20036142608013C19
:1008F000031C8F2C031D802C2508683C031C8F2CA7
:100900000E302502B7002608B8000130031C023063
:10091000B802A030370784000008B300B6142608D8
:10092000013C031CA82C031D992C25080E3C031C1C
:10093000A82C25080E3CB7000130B8002608031C7F
:10094000260FB802A030370784000008B300B610A5
:10095000A608031DBE2C2508B43C031CBE2C5A302F
:100960002502B7002608B8000030031C0130B80289
:10097000A030370784000008B300B610A608031D96
:10098000D32C25085A3C031CD32C25085A3CB7000D
:10099000B8012608031C260FB802A03037078400D0
:1009A0000008B300B6148A11E82D2030A000A00B77
:1009B000D72CDA2C0000A410240883168700831299
:1009C00087142030A000A00BE32CE62C0000A4101C
:1009D000240883168700831287102030A000A00B04
:1009E000EF2CF22C00000800AB012B08023C031C8A
:1009F000132D2B08023CB7002908A0003708A100DE
:100A00000319062D0310A00CA10B022D20180A2D8E
:100A100007110B2D07152411240883168700831254
:100A2000D524AB0AF52C0800AB012B08073C031CAE
:100A3000332D2B08073CB7002A08A0003708A10077
:100A40000319262D0310A00CA10B222D20182A2DEE
:100A500007112B2D071524112408831687008312F4
:100A6000D524AB0A152D080024102408831687000E
:100A700083120710A901F4243308AA001425F424D2
:100A80003508AA0014252410240883168700831231
:100A900007144230A000A00B4B2D000024102408A6
:100AA00083168700831207100130A900F42432084E
:100AB000AA001425F4243408AA00142524102408BC
:100AC00083168700831207144230A000A00B662D06
:100AD00000002410240883168700831207100230B8
:100AE000A900F4243208AA001425F4243408AA002A
:100AF000142524102408831687008312071442301B
:100B0000A000A00B812D000024102408831687006C
:100B1000831207100330A900F4243308AA00142517
:100B2000F4243508AA00142524102408831687000D
:100B3000831207148A11E92D003036190130B700ED
:100B40003718A42D8810A52D88148316881000301E
:100B50008312B6190130B7003718B02D0811B12D26
:100B60000815831608110030831236180130B700BB
:100B70003718BC2D8711BD2D8715A41124088316A5
:100B8000870000308312B6180130B7003718CA2D1D
:100B90000810CB2D08148316081083128A11E52D36
:100BA00003081F398300FF30A40083161F149F140D
:100BB0001F159F111F149F101F159F1583121F13C0
:100BC0009F1783169F1783121F140A29F729C02A1B
:080BD000342D9C2DE52D63007E
:02400E00723FFF
:00000001FF
